:100000000C949F040C94BC040C94B30B0C94BC048F
:100010000C94BC040C94BC040C94B30B0C94BC0462
:100020000C94BC040C94BC040C94BC040C94BC0450
:100030000C94BC040C94BC040C94BC040C94BC0440
:100040000C94B40B0C94BC040C94BC040C94BC0431
:100050000C94BC040C94BC040C94BC040C94BC0420
:100060000C94BC040C94BC0453687574646F776E74
:100070002E2E2E00207777772E6F626475696E6F53
:100080002E636100204F424475696E6F204C697485
:1000900065004672656465726963204C616D6F72BC
:1000A0006365002020202028632920323031300071
:1000B00025387300252D38730025732025636900CA
:1000C0002D2025642563202B200025732025730017
:1000D00025732025630025642025730025642025D1
:1000E00063002573202525002564052563002573FD
:1000F0002056002564206B5061002530336C64006D
:100100002530326C6400256C64001010190204095B
:10011000010100000000001B1B1B10141814001F1D
:100120001515020408100404070507050700000060
:1001300000001F1515000E04040E02040810070429
:1001400005073C5945533E206E6F200020796573AA
:10015000203C4E4F3E0053637220257520636F7222
:100160006E657220257500436F6E66696720736344
:100170007265656E3F0050656E64696E6720445419
:100180004300416476616E63656420736C656570DD
:1001900000456E67696E65206473706C636D6E7484
:1001A000002D202564644C202B20004469737420AA
:1001B00061646A757374004675656C2061646A7564
:1001C00073740054616E6B2073697A6500436F6EBF
:1001D0006669672073657474696E67733F0044696C
:1001E00073706C61792064656C6179002D202564E1
:1001F0006D73202B20004675656C2F686F7572201B
:100200007370656564002D202564256304202B2010
:1002100000557365206D657472696320756E69742D
:1002200073004C434420636F6E74726173740043B7
:100230006F6E66696720646973706C61793F005204
:100240006573657420747269702064617461005212
:10025000657365742074616E6B2064617461005015
:10026000494420537570706F72743030004D494CA2
:1002700020436F6465202020202000467265657A47
:100280006520445443202020004675656C2053743B
:1002900061747573202000456E67696E65204C6F30
:1002A0006164202000436F6F6C616E742054656D33
:1002B000702000535446542042616E6B2031202040
:1002C000004C5446542042616E6B20312020005374
:1002D0005446542042616E6B20322020004C54461C
:1002E000542042616E6B20322020004675656C20E0
:1002F0005072657373757265004D616E69666F6CDF
:1003000064205072657300456E67696E65205250B7
:100310004D2020200056656869636C652053706528
:1003200065640054696D696E67204164766E63652B
:1003300000496E74616B652054656D702020004D1E
:100340006173732041697220466C6F770054687244
:100350006F74746C6520506F732000536563204187
:100360006972207374617420004F322053656E737C
:100370006F72732031200042315331204F322056AA
:100380006F6C74200042315332204F3220566F6C14
:1003900074200042315333204F3220566F6C74204A
:1003A0000042315334204F3220566F6C742000428B
:1003B000325331204F3220566F6C7420004232533A
:1003C00032204F3220566F6C74200042325333205B
:1003D0004F3220566F6C74200042325334204F321B
:1003E00020566F6C7420004F4244205374616E6439
:1003F00061726420004F322053656E736F727320F8
:100400003220004175786C727920496E70757420C5
:100410000052756E74696D6520537461727400507A
:10042000494420537570706F7274323000446973A0
:1004300074204D494C204F6E2020004675656C207D
:100440005261696C20507273004675656C20526170
:10045000696C2044736C004F325331205752205640
:100460006F6C7420004F32533220575220566F6CFD
:100470007420004F32533320575220566F6C742033
:10048000004F32533420575220566F6C7420004F67
:1004900032533520575220566F6C7420004F325320
:1004A0003620575220566F6C7420004F325337203D
:1004B000575220566F6C7420004F325338205752D9
:1004C00020566F6C742000436F6D6D616E64204523
:1004D0004752202000454752204572726F722020FB
:1004E000202000436F6D6D616E6420457661702041
:1004F000004675656C204C6576656C202020004EAA
:1005000062205761726D205570732020004469731A
:1005100074204D494C20436C722000457661702058
:100520005072657373757265004261726F2050720C
:10053000657373757265004F3253312057522043F3
:1005400075727220004F3253322057522043757219
:100550007220004F3253332057522043757272205D
:10056000004F325334205752204375727220004F8F
:10057000325335205752204375727220004F325348
:1005800036205752204375727220004F3253372065
:100590005752204375727220004F32533820575201
:1005A0002043757272200042315331204361742020
:1005B00054656D700042325331204361742054659C
:1005C0006D700042315332204361742054656D7068
:1005D0000042325332204361742054656D700050E4
:1005E000494420537570706F72743430004D6F6ED3
:1005F00069746F722053746174200045434D205616
:100600006F6C746167652020004162736F6C757454
:1006100065204C6F616400436D6420457175205204
:100620006174696F0052656C617469766520546805
:10063000727400416D6269656E742054656D70203E
:1006400000416273205468727420506F73420041FD
:100650006273205468727420506F73430041636367
:100660006C2050646C20506F7344004163636C20B5
:1006700050646C20506F7345004163636C2050647C
:100680006C20506F73460054687274204163747517
:1006900061746F720054696D65204D494C204F6E36
:1006A00020200054696D65204D494C20436C722018
:1006B000004D61782056616C756520233120004D16
:1006C00061782056616C756520233220004675657F
:1006D0006C20547970652020202000457468616E7C
:1006E0006F6C202520202020004E6F2044697370FD
:1006F0006C617920202000496E7374616E74204310
:100700006F6E73200041766720436F6E73205461D3
:100710006E6B004675656C205573652054616E6B79
:100720000044697374616E63652054616E6B005799
:1007300061737465642054616E6B20200041757490
:100740006F6E6F6D792054616E6B00417667204348
:100750006F6E73204F757420004675656C2055735D
:1007600065204F7574200044697374616E63652061
:100770004F75742000576173746564204F75742041
:100780002020004261747465727920566F6C742069
:10079000004F42443243415242004F42444550418F
:1007A0000000004F42444550412632004F42443140
:1007B00000000000004E4F204F4244000000454F13
:1007C00042440000000000454F4244263200000031
:1007D000454F42442645504100452645504126326A
:1007E00000004A4F424400000000004A4F424426A5
:1007F000320000004A26454F42440000004A264588
:100800004F42442632004555524F34423100004594
:1008100055524F35423200004555524F204300009B
:1008200000454D440000000000002563253032588B
:10083000253032582000256420494E20454355007C
:1008400050454E44494E4720434F44453A004641A7
:10085000554C5420434F44453A00256C58002573AD
:10086000206B5061004F42443A25303258002564D5
:1008700005002564206D696E0025753A25303275B6
:100880003A253032750025730025646D562F256496
:100890002525002530345800434C2D4661756C7475
:1008A000004F4C2D4661756C74004F4C2D4472699D
:1008B000766500434C004F4C00257320672F730072
:1008C00025642052504D0025303258204E2F4100D3
:1008D000253032583A25730025733A2530325800B6
:1008E000FD00000000000000C6CAF1000008000082
:1008F0000008000000080000FF000000FFEBFF0000
:10090000323962697473003131626974730032354F
:10091000306B2F003530306B2F0043414E20496E35
:1009200069742E2E2E0004B6E704B6D304B6C704AD
:10093000B6C302900703AC0103AC0002900011247F
:100940001FBECFEFD4E0DEBFCDBF11E0A0E0B1E02D
:10095000E0E9FBE302C005900D92A634B107D9F798
:1009600011E0A6E4B1E001C01D92A63AB107E1F79B
:100970000E94600A0C94C61D0C9400002F923F92B6
:100980004F925F926F927F928F929F92AF92BF929F
:10099000CF92DF92EF92FF920F931F93DF93CF934B
:1009A000CDB7DEB7AA970FB6F894DEBF0FBECDBFA6
:1009B0000E94070C20916101309162014091630116
:1009C00050916401621773078407950778F41B013F
:1009D0002C01221A330A440A550A29EB39E44CE067
:1009E00052E0220E331E441E551E06C01B012C0170
:1009F000221A330A440A550A609361017093620116
:100A000080936301909364018E010F5F1F4FB801C3
:100A10008DE00E94BB127AA769A777FD41C1B8019A
:100A200081E10E94BB128B0177FD3AC180910001E8
:100A300090E00817190714F4009300015E01089470
:100A4000A11CB11CB5018CE00E94BB126B017C01A2
:100A500097FD26C1B50183E00E94BB129B01AC014A
:100A600089A59AA5892B49F08091000190E005960F
:100A70008017910714F032FD05C0C114D104E104C0
:100A8000F10461F4E7E7F1E01192119291E0E739A6
:100A9000F907D1F76624772443013EC08E010F5F2A
:100AA0001F4FB80180E10E94BB123B014C0197FF30
:100AB00033C0B8018BE00E94BB125B0177FDF0C030
:100AC000B8018FE00E94BB128B0177FDE9C0B50130
:100AD000882777FD8095982FA70196010E942D1AEF
:100AE0000F5E1E4F9801442737FD4095542F0E94FA
:100AF000951ACA01B9012091090130E040E050E0A7
:100B00000E942D1A25E030E040E050E00E94951A46
:100B1000C901DA013C014D018091080190E029A54D
:100B20003AA5289FB001299F700D389F700D1124A0
:100B3000882777FD8095982FA20191010E942D1A98
:100B400020E13EE040E050E00E94731A59016A0142
:100B50002091070130E040E050E0C401B3010E9461
:100B60002D1AA20191010E942D1A2EE233EA41E0D2
:100B700050E00E94731A79018A0180910C019091D2
:100B80000D01A0910E01B0910F018A0D9B1DAC1DAE
:100B9000BD1D80930C0190930D01A0930E01B093A5
:100BA0000F018091100190911101A0911201B0915B
:100BB00013018E0D9F1DA01FB11F809310019093F4
:100BC0001101A0931201B093130149A55AA5452B19
:100BD000A1F48091140190911501A0911601B0919A
:100BE00017018E0D9F1DA01FB11F809314019093BC
:100BF0001501A0931601B0931701809118019091EF
:100C00001901A0911A01B0911B01A80EB91ECA1EAC
:100C1000DB1EA0921801B0921901C0921A01D09265
:100C20001B0180911C0190911D01A0911E01B091AA
:100C30001F018E0D9F1DA01FB11F80931C0190935B
:100C40001D01A0931E01B0931F0189A59AA5892BB0
:100C5000A1F48091200190912101A0912201B091F5
:100C60002301E80EF91E0A1F1B1FE0922001F092DB
:100C70002101009322011093230180914701E82F65
:100C8000F0E0DF01A959BE4F99A59C93EE0FFF1F1D
:100C9000E958FE4F718260828F5F8F7080934701A9
:100CA000AA960FB6F894DEBF0FBECDBFCF91DF91ED
:100CB0001F910F91FF90EF90DF90CF90BF90AF907A
:100CC0009F908F907F906F905F904F903F902F906C
:100CD0000895EF92FF920F931F93DF93CF93CDB7B9
:100CE000DEB760970FB6F894DEBF0FBECDBF7C01B4
:100CF00080E40E945D0C2CE130E0AC01429FC00119
:100D0000439F900D529F900D112464E670E00E9465
:100D10004C1A80E090E021E08E010F5F1F4FA80188
:100D20000E945D0B1F930F938EEE90E09F938F9325
:100D3000FF92EF920E94E61A8DB79EB706960FB605
:100D4000F8949EBF0FBE8DBF60960FB6F894DEBFBD
:100D50000FBECDBFCF91DF911F910F91FF90EF900C
:100D600008958F929F92AF92BF92CF92DF92EF92AF
:100D7000FF920F931F93DF93CF93CDB7DEB76097AA
:100D80000FB6F894DEBF0FBECDBF4C018CE0689F5C
:100D9000F0011124E45FFE4FA480B580C680D780A7
:100DA000E080F1800281138187E3A81689E8B80604
:100DB00081E4C80680E0D806C8F497E3E91699E80C
:100DC000F90691E4090790E0190780F4C601B5011E
:100DD00028EE33E040E050E00E942D1A5B016C01E8
:100DE000C801B7010E942D1A7B018C01C801B7010F
:100DF00028EE33E040E050E00E94731A79018A0146
:100E0000E114F1040105110529F0A114B104C10494
:100E1000D10451F480910301882319F460E070E05B
:100E200019C066E077E216C0C601B501A8019701B6
:100E30000E94731AB90180910301882359F4232B6E
:100E400049F040E050E06EEC76E983E090E00E94EB
:100E5000731AB90170939B0160939A014091030149
:100E60004F5F87E26730780718F066E077E204C0EA
:100E700093E0683E790730F04150CB016AE070E0C2
:100E80000E944C1A80E090E0242F8E010F5F1F4FCC
:100E9000A8010E945D0B83E591E09F938F931F93C0
:100EA0000F938AEC90E09F938F939F928F920E9472
:100EB000E61A8DB79EB708960FB6F8949EBF0FBE80
:100EC0008DBF60960FB6F894DEBF0FBECDBFCF9139
:100ED000DF911F910F91FF90EF90DF90CF90BF9027
:100EE000AF909F908F900895AF92BF92CF92DF9274
:100EF000EF92FF920F931F93CF93DF93EC018091BA
:100F00000601282F30E040E050E080910301882363
:100F100031F4CA01B9010E94210B9B01AC01CA0145
:100F2000B90128EE33E040E050E00E942D1A7B0129
:100F30008C016091100170911101809112019091CA
:100F400013010E94731A59016A01EA14FB040C058B
:100F50001D0550F1A114B104C104D10429F1EA180E
:100F6000FB080C091D0960910C0170910D01809125
:100F70000E0190910F01A60195010E94731AC801FC
:100F8000B7010E942D1A20EA36E841E050E00E94A5
:100F9000731A80910301882349F4B90180E090E03D
:100FA0000E944E0B9B0102C020E030E08091500176
:100FB00090E09F938F933F932F938CED90E09F93BE
:100FC0008F93DF93CF930E94E61A8DB79EB7089652
:100FD0000FB6F8949EBF0FBE8DBFDF91CF911F91CA
:100FE0000F91FF90EF90DF90CF90BF90AF9008955A
:100FF000EF92FF920F931F93DF93CF93CDB7DEB79E
:1010000060970FB6F894DEBF0FBECDBF7C0170E0D5
:10101000FB01EE0FFF1FE60FF71FEE0FFF1FEE0F96
:10102000FF1FEE5FFE4F628573858485958520E105
:1010300037E240E050E00E94731A622FE42F952FB0
:1010400080910301882331F4732F842F0E944E0B6B
:10105000372FE82F21E08E010F5F1F4FA801732F5C
:101060008E2F0E945D0B8091500190E09F938F9393
:101070001F930F9380ED90E09F938F93FF92EF92D9
:101080000E94E61A8DB79EB708960FB6F8949EBFD9
:101090000FBE8DBF60960FB6F894DEBF0FBECDBFFA
:1010A000CF91DF911F910F91FF90EF900895CF9214
:1010B000DF92EF92FF920F931F93DF93CF93CDB701
:1010C000DEB760970FB6F894DEBF0FBECDBF6C01E0
:1010D0007901CB01BA0120E137E240E050E00E9403
:1010E000731A622FE42F952F80910301882331F426
:1010F000732F842F0E94300B372FE82F22E08E01B0
:101100000F5F1F4FA801732F8E2F0E945D0B8091E0
:10111000560190E09F938F931F930F93FF92EF924E
:10112000DF92CF920E94E61A8DB79EB708960FB64F
:10113000F8949EBF0FBE8DBF60960FB6F894DEBFC9
:101140000FBECDBFCF91DF911F910F91FF90EF9018
:10115000DF90CF90089570E0FB01EE0FFF1FE60FC8
:10116000F71FEE0FFF1FEE0FFF1FEE5FFE4F4289CE
:1011700053896489758929EB30E00E9457080895E6
:1011800070E0FB01EE0FFF1FE60FF71FEE0FFF1FD2
:10119000EE0FFF1FEA5FFE4F42855385648575851C
:1011A00020ED30E00E94570808958F929F92AF92F1
:1011B000BF92CF92DF92EF92FF920F931F93DF9334
:1011C000CF93CDB7DEB760970FB6F894DEBF0FBEF2
:1011D000CDBF4C01E7E6F1E047E751E0AA24BB248C
:1011E000EE24FF248701DD248081A80EB11CDA01E2
:1011F0002D913C91C901A0E0B0E0E80EF91E0A1F54
:101200001B1F232B09F0D39431964E5F5F4FB1E043
:10121000E737FB0749F7DD20A9F02091070130E00F
:1012200040E050E0B701C8010E942D1A24E6D29E8A
:101230009001112440E050E00E94731AC901DA01C4
:101240007C018D0184E0B694A7948A95E1F78091A2
:101250000401682F70E080910301882321F480E06D
:1012600090E00E943F0B6A157B0538F0B0E1CB2E71
:10127000B7E2DB2EBB24B3940BC08091080190E051
:10128000A89E6001A99ED00CB89ED00C1124BB244E
:10129000C801B7012BE13DE040E050E00E942D1A6B
:1012A000960140E050E00E94731AB9018091030159
:1012B0008823A9F4BB2029F080E090E00E94300B45
:1012C0000EC0232B19F466E077E209C040E050E03D
:1012D0006EEC76E983E090E00E94731AB901709396
:1012E00098016093970180910301882321F4BB202A
:1012F00011F441E001C042E087E26730780718F05E
:1013000066E077E204C093E0683E790730F0415030
:10131000CB016AE070E00E944C1A80E090E0242F3C
:10132000AE014F5F5F4F0E945D0BBB2019F483E558
:1013300091E002C086E591E09F938F93CE010196E4
:101340009F938F938AEC90E09F938F939F928F92BD
:101350000E94E61AADB7BEB718960FB6F894BEBF96
:101360000FBEADBF8B2D60960FB6F894DEBF0FBEDB
:10137000CDBFCF91DF911F910F91FF90EF90DF9044
:10138000CF90BF90AF909F908F900895FB01803ECB
:1013900021F480E2808311820895813E21F4CB0103
:1013A0000E94D5080895823E11F460E015C0833E86
:1013B00011F460E018C0843E11F460E01BC0853E6B
:1013C00011F460E01EC0863E21F4CB010E94740738
:1013D0000895873E29F461E0CF010E94B106089587
:1013E000883E29F461E0CF010E94C0080895893E3B
:1013F00029F461E0CF010E94F80708958A3E29F49C
:1014000061E0CF010E94AB0808958B3E21F4CB012F
:101410000E94690608950E94BB1208950F931F93BE
:10142000DF93CF93CDB7DEB7C055D0400FB6F89459
:10143000DEBF0FBECDBF082F862F1982BE016F5FA2
:101440007F4F0E94C6098981882371F1002321F012
:10145000023011F088E001C080E060E0023008F066
:1014600061E00E94070D002329F0023019F020EB03
:1014700030E002C024EB30E0CE0101969F938F93C1
:101480003F932F938E01075D1F4F1F930F930E9471
:10149000E61AC8010E94590D8DB79EB706960FB681
:1014A000F8949EBF0FBE8DBFC05BDF4F0FB6F894A0
:1014B000DEBF0FBECDBFCF91DF911F910F91089579
:1014C000CDB7DEB7A897DEBFCDBF0E94330C0E9418
:1014D000D91084E291E090936601809365011092A7
:1014E0009C0110E07E010894E11CF11C01C011E098
:1014F0000E94070C60936101709362018093630105
:1015000090936401109299010E94A10D112361F43E
:1015100083EA90E00E94870D82E990E00E944D0DE1
:1015200088EE93E00E941F0C84E890E00E94870DF3
:1015300084E790E00E944D0D88EE93E00E941F0C1E
:10154000112321F40E945E160E94781581E00E940A
:10155000A00EE7E6F1E0119221E0E737F207D9F7B4
:10156000E7E7F1E01192119281E0E739F807D1F74E
:1015700080910B01882319F087E00E94A011B70128
:1015800081E00E94BB1297FF07C083E00E94A01178
:10159000882311F00E949F1180919C010E94790D77
:1015A0000E94BE04E0916501F0916601608180E0D7
:1015B0000E940E0AE0916501F0916601618181E06F
:1015C0000E940E0AE0916501F0916601628182E05D
:1015D0000E940E0AE0916501F0916601638183E04B
:1015E0000E940E0A80910501882319F090E00E9464
:1015F0001F0C0E940D1080919901853088F20E9485
:101600001E1188E690E00E94870D80ED97E00E9411
:101610001F0C0E94920D80910A010E94830C84E6A7
:1016200090E00E941F0C80910A01882309F05FCF8F
:10163000B7010E94BB126F5F7F4F8F4F9F4F59F3CF
:1016400056CF2AE731E040E050E00E942D1A24E610
:1016500030E040E050E00E94731ACA01B9010895D9
:1016600024E630E040E050E00E942D1A2AE731E005
:1016700040E050E00E94731ACA01B901089529E4BC
:1016800036E040E050E00E942D1A28EE33E040E0C2
:1016900050E00E94731ACA01B901089528EE33E0A0
:1016A00040E050E00E942D1A29E436E040E050E08E
:1016B0000E94731ACA01B90108951F93CF93DF9353
:1016C000EA01122F2223A9F49F938F937F936F93A4
:1016D00086E091E09F938F935F934F930E94E61A69
:1016E0008DB79EB708960FB6F8949EBF0FBE8DBFFC
:1016F00036C0213039F49F938F937F936F9380E0AE
:1017000091E008C02230A1F49F938F937F936F9351
:101710008AEF90E09F938F93DF93CF930E94E61A16
:101720008DB79EB708960FB6F8949EBF0FBE8DBFBB
:1017300060E170E0CE010E94DB1A982F9F5F20E0ED
:10174000FE01E90FF11D82913196808391502F5F48
:101750001217B0F7C90FD11D8091A1018883DF91C5
:10176000CF911F91089518951F920F920FB60F9267
:1017700011242F933F938F939F93AF93BF933091F7
:10178000480183B129B120788370282B2095232725
:1017900080914F018223809580934F0190914E015B
:1017A0009223982790934E0182238923982F932781
:1017B00090934801982380914901892B8093490196
:1017C00080914A0190914B01A0914C01B0914D0143
:1017D0000196A11DB11D80934A0190934B01A093E6
:1017E0004C01B0934D01BF91AF919F918F913F916B
:1017F0002F910F900FBE0F901F901895F894909115
:10180000490189239827909349017894089560911C
:101810004A0170914B0180914C0190914D0127E05C
:10182000660F771F881F991F2A95D1F72DE730E0A3
:1018300040E050E00E94731ACA01B901089523B72D
:10184000217F23BF9C012F5F3F4F09C083B7816079
:1018500083BF889583B78E7F83BF21503040211589
:101860003105A1F7089514BE88E10FB6F89480936E
:101870006000109260000FBE789483E085BD91E017
:1018800090936E0087E880937A0080E480937C00D8
:101890002198299A2098289A57985F9A5098589A90
:1018A0005198599A8AEC8093640080E880BF8FE356
:1018B00080937E0090937F00089580937C0083B78F
:1018C000817F83BF83B7816083BF889583B78E7F15
:1018D00083BF83B7816083BF889583B78E7F83BFC3
:1018E00080917A00806480937A0080917A0086FDEE
:1018F000FCCF9091780080917900382F20E0290F5B
:10190000311DC90108951F93182F83B7817F84600B
:1019100083BF80917A008F7780937A00F8941123A7
:1019200039F01092690082E08DBB0E946C1808C0EB
:10193000A89514BE88E18093600087E480936000DE
:1019400083B7816083BF7894889583B78E7F83BF88
:10195000112321F01DBA0E94591808C088E10FB662
:10196000F89480936000109260000FBE80917A001E
:10197000806880937A0010924A0110924B01109275
:101980004C0110924D011F91089587FF02C0459AA6
:1019900001C0459886FF02C0449A01C0449885FF63
:1019A00002C0439A01C0439884FF02C0429A08953E
:1019B00042980895419A85E0982F9A95F1F74198B9
:1019C0008A95F1F708950F931F93082F0E94C50C75
:1019D000419A15E0812F8A95F1F74198812F8A95D8
:1019E000F1F7802F8295807F0E94C50C419A812F4C
:1019F0008A95F1F741981A95F1F78AEC8A95F1F7F3
:101A00001F910F9108955C980E94E30C08958058EF
:101A10006111805C0E94030D08955C9A0E94E30CA2
:101A20000895EF92FF920F931F93E62E142F052F28
:101A3000880F880F880F805C0E94030DEE0CEE0C5F
:101A4000EE0C812F902FFC018F01FF2407C0F801BD
:101A500084910E940D0DF3940F5F1F4FFE14B8F395
:101A60001F910F91FF90EF9008951F9310E080E277
:101A70000E940D0D1F5F1031D1F71F910895CF9374
:101A8000DF93EC0102C00E940D0DFE0121968491AE
:101A90008823C9F7DF91CF9108950F931F938C018D
:101AA00080EC0E94030DC8010E943F0D1F910F9111
:101AB0000895CF93DF93EC0102C00E940D0D899130
:101AC0008823D9F7DF91CF9108950F931F938C014D
:101AD00080EC0E94030DC8010E94590D1F910F91C7
:101AE000089581E00E94030D82E090E00E941F0CA7
:101AF00008951F93182F0E94710D112331F44AE0AD
:101B000051E067E081E00E94110D1F9108950F934D
:101B10001F938C010E94710DC8010E943F0D1F91FF
:101B20000F91089514BC5D985E9841985C98429816
:101B300043984498459882E090E00E941F0C5A9880
:101B40000895FF920F931F93529A5A9A83EA84BD85
:101B5000809101012FE3829FC001112488BD8091F3
:101B6000020187BD559A569A399A549A3A9A3B9AE5
:101B70003C9A3D9A80E190E00E941F0C10E005E045
:101B800080E30E94C50C419A85E0F82E802F8A954B
:101B9000F1F74198802F8A95F1F785E090E00E9457
:101BA0001F0C1F5F133061F780E20E94C50C419A41
:101BB0008F2D8A95F1F741988F2D8A95F1F781E065
:101BC00090E00E941F0C88E20E94030D8CE00E94AE
:101BD000030D86E00E94030D0E94710D1F910F916D
:101BE000FF90089582E00E94FE0B80939D0181E0AA
:101BF0000E94FE0B80939F0180E80E94FE0B809361
:101C00009E0108958AEF90E00E941F0C0E94F20D41
:101C10000E94BE0408957F928F929F92AF92BF92CE
:101C2000CF92DF92EF92FF920F931F93DF93CF93A8
:101C3000CDB7DEB7A8970FB6F894DEBF0FBECDBF05
:101C40004B015A01122F702EDE2C0E94870D012F9E
:101C500010E07E010894E11CF11C80919D01882315
:101C600031F0F5018081871511F08C1909C0809140
:101C70009E01882331F0F50180818D1511F08C0DC6
:101C8000808384EC0E94030D1F930F93F5018081E4
:101C900090E09F938F939F928F92FF92EF920E947A
:101CA000E61AC7010E94590D8091020187BD0E946A
:101CB000020E8DB79EB708960FB6F8949EBF0FBE62
:101CC0008DBF80919F01882341F2A8960FB6F894AA
:101CD000DEBF0FBECDBFCF91DF911F910F91FF905F
:101CE000EF90DF90CF90BF90AF909F908F907F90BC
:101CF00008951F93182F10929E0110929F01109229
:101D00009D0180919D01882311F011E004C0809114
:101D10009E01811110E083EC0E94030D112319F440
:101D20008CE491E002C082E491E00E943F0D0E94A9
:101D3000020E80919F01882321F3812F1F91089526
:101D40001F93182F813071F0882319F48FE492E0EB
:101D500002C08FE392E00E94870D80E00E94790E1E
:101D6000813091F4ECE01E9FF0011124E45FFE4FFE
:101D700010821182128213821482158216821782B7
:101D800010861186128613860E94710D1F91089588
:101D90006F927F928F929F92AF92BF92CF92DF927B
:101DA000EF92FF920F931F93DF93CF93CDB7DEB7E0
:101DB000A8970FB6F894DEBF0FBECDBF80E00E949B
:101DC000790D8FE292E00E94870D80E00E94790EEB
:101DD0008823A9F1EAE0CE2E74E6E72E00E025E2A2
:101DE00042E051E060EC70E082E292E00E940B0E73
:101DF00081E192E00E94870D809103010E94790E9B
:101E0000809303010E94B210CC24C394EE24EA9480
:101E10002091500144E051E066E072E086EF91E0ED
:101E20000E940B0E62E3C62E5AEFE52E20E045E03D
:101E300051E06CEE71E08EED91E00E940B0E8DECA6
:101E400091E00E94870D80E00E94790E882309F4BA
:101E500044C0CC24C394EE24EA9401E020915601BE
:101E600046E051E060EC70E083EC91E00E940B0EE4
:101E700025E247E051E060EC70E087EB91E00E94E2
:101E80000B0E25E248E051E060EC70E08BEA91E057
:101E90000E940B0E60E080E10E943B11882349F410
:101EA00020E049E051E061EA71E081E991E00E94BF
:101EB0000B0E82E891E00E94870D80910A010E943A
:101EC000790E80930A0186E791E00E94870D809148
:101ED0000B010E94790E80930B0187E691E00E942E
:101EE000870D80E00E94790E882309F47BC080E092
:101EF00090E046E5642E41E0742E4E010894811C6A
:101F0000911C5FC00E94710DDF92CF92BF92AF9281
:101F10007F926F929F928F920E94E61AC4010E9454
:101F2000590DF701008110E02DB73EB7285F3F4FF4
:101F30000FB6F8943EBF0FBE2DBF80919D01882340
:101F400041F0015061E0802F0E943B118823C9F3CA
:101F500062C080919E01882341F00F5F61E0802F75
:101F60000E943B118823C9F356C0143040F440E06E
:101F7000602FC4010E94C4150E94650D09C0B40100
:101F8000802F0E94C609C4010E94650D0E94350D74
:101F90000E94020E80919F01882319F41F5F177021
:101FA000CCCFF70101937F010894C11CD11CF5E04F
:101FB000CF16D10409F0A6CF22E0A216B10491F009
:101FC000C5017C01EE0CFF1CEE0CFF1CE4E2F1E00D
:101FD000EE0EFF1E21E0C22ED12C5C010894A11C44
:101FE000B11C90CF80919C010E94790DA8960FB6EC
:101FF000F894DEBF0FBECDBFCF91DF911F910F913F
:10200000FF90EF90DF90CF90BF90AF909F908F9018
:102010007F906F90089510E0AACFEF92FF921F93E8
:10202000DF93CF93CDB7DEB7A8970FB6F894DEBF96
:102030000FBECDBF0E94F20D90919F01992341F0F8
:1020400080919D01882321F080E00E94A00E7EC037
:1020500080919D01882309F461C08091460190E040
:1020600001968170907080934601880F991F880FA8
:10207000991F8C5D9E4F909366018093650110922D
:102080009C0180E00E94790D10E07E010894E11C23
:10209000F11C0E94710DE0916501F091660180E0F4
:1020A00090E0112311F081E090E0E80FF91F412F3B
:1020B0006081C7010E94C4150E94590DE09165011D
:1020C000F0916601112319F083E090E002C082E0F4
:1020D00090E0E80FF91F412F6081C7010E94C415ED
:1020E0000E94650D0E94020E80919D01882371F46B
:1020F0000E94020E80919D01882341F40E94020EED
:1021000080919D01882311F40E94020E80919D010F
:102110008823E1F41F5F1230C9F0BBCF80919E018C
:10212000882381F08091010190E0019665E070E0E4
:102130000E94601A809301012FE3829FC001112445
:1021400088BD04C0992311F00E94C80EA8960FB64E
:10215000F894DEBF0FBECDBFCF91DF911F91FF90EE
:10216000EF90089580910301882389F083E08093A4
:10217000500181E08093530182E0809354018CE40C
:102180008093560183E48093A0018CE20FC086E027
:10219000809350018093530187E08093540187E43A
:1021A0008093560186E48093A0018EE28093A10182
:1021B00008950F931F93DF93CF93CDB7DEB7AA9700
:1021C0000FB6F894DEBF0FBECDBF4AE250E060E02C
:1021D00070E08E010F5F1F4FC8010E94E21C8AE26F
:1021E00090E00E94F21CAC0120E030E0F801BE015A
:1021F000655D7F4F8191280F311DE617F707D1F7F5
:102200004217530749F4A2E0B1E0FE0131968AE299
:1022100001900D928150E1F784E080935101809309
:1022200057010E94B210AA960FB6F894DEBF0FBEF7
:10223000CDBFCF91DF911F910F910895CF93DF9381
:10224000C0E0D0E0E2E0F1E08191C80FD11D81E073
:10225000EC32F807C9F74AE250E060E070E0CF01E5
:102260008A970E94F81CBE018AE290E00E94101D2D
:10227000DF91CF910895982F882309F45BC08132B4
:10228000B8F460E080E2891B21E030E040E050E0FB
:1022900004C0220F331F441F551F8A95D2F7809127
:1022A000A2019091A301A091A401B091A50131C018
:1022B0008134B8F460E080E4891B21E030E040E044
:1022C00050E004C0220F331F441F551F8A95D2F7D8
:1022D0008091590190915A01A0915B01B0915C01EC
:1022E00018C0813600F560E080E6891B21E030E00F
:1022F00040E050E004C0220F331F441F551F8A9551
:10230000D2F780915D0190915E01A0915F01B09143
:102310006001282339234A235B2321153105410518
:10232000510559F007C0662339F0803E28F060E07F
:102330008C3E18F461E001C060E0862F0895089596
:102340002F923F924F925F926F927F928F929F92C5
:10235000AF92BF92CF92DF92EF92FF920F931F93B3
:10236000DF93CF93CDB7DEB7C852D1400FB6F89404
:10237000DEBF0FBECDBF182F833019F0873009F0B4
:10238000DEC0812F0E943316CE0189960E942C1741
:1023900097FDD5C029A530E0812F90E0805C9F4F4C
:1023A0002817390709F0CBC0AAA4AA2009F4C8C08D
:1023B000133019F48EE498E002C080E498E00E94A3
:1023C000870D8A2C99249F928F9286E398E09F93A1
:1023D0008F932E010894411C511C5F924F920E94D2
:1023E000E61AC2010E94650D80ED97E00E941F0C65
:1023F000CC24DD248DB79EB706960FB6F8949EBF09
:102400000FBE8DBF14010E94710DCC2019F08DE21A
:102410000E940D0D82E80E94030DEC2CFF24870121
:102420000F5F1F4F000F111FE9E2F0E0EC0FFD1FDF
:102430000E0F1F1FBB243701E214F30408F046C03F
:10244000F8013081832F807C11F420E509C086FFDC
:1024500002C023E405C087FD02C025E501C022E4D7
:10246000F801818190E09F938F93832F90E08F7389
:1024700090709F938F93822F90E09F938F938AE227
:1024800098E09F938F93E1E0F0E0EC0FFD1FFF9346
:10249000EF930E94E61AC2010E94590D8DB79EB7B4
:1024A0000A960FB6F8949EBF0FBE8DBF91E0B91685
:1024B00019F482EC0E94030DB3940894E11CF11C02
:1024C0000E5F1F4FE4E0BE1609F0B6CF83010C5F2C
:1024D0001F4F081519051CF48BE20E940D0D0E9478
:1024E000020E80919D01882329F480919E0188230A
:1024F00049F406C0CC2031F0FCEFCF0EDD2417C02C
:10250000D39401C0DD2480919E01882349F00815F1
:10251000190534F484E6D81691F094E0C90E07C08A
:10252000E4E6DE1661F080919F018823C1F280917C
:102530009F01882309F467CFF4E6DF1609F4AA2483
:102540008A2DC85DDE4F0FB6F894DEBF0FBECDBF3B
:10255000CF91DF911F910F91FF90EF90DF90CF907F
:10256000BF90AF909F908F907F906F905F904F90B3
:102570003F902F900895AF92BF92CF92DF92EF924B
:10258000FF920F931F93DF93CF93CDB7DEB7A09742
:102590000FB6F894DEBF0FBECDBF082F5B011091C0
:1025A000030160E00E943B11882389F4802F90E0B2
:1025B0009F938F9387EC98E09F938F93BF92AF92F6
:1025C0000E94E61ACC24CA94DC2C760154C2602FF7
:1025D00081E00E942516CE0101960E942C17AC01C5
:1025E00097FD06C08981813419F42A81201751F0A2
:1025F000809199018F5F80939901CC24CA94DC2C3F
:10260000760163C210929901AE81BD819C817B816C
:10261000E92FF72F6F01EE24FF242C3061F472E0D4
:10262000F594E794D794C7947A95D1F7DF92CF9237
:1026300080EC98E01AC2203171F48E010F5E1F4FBA
:1026400022E0A801C701B6010E945D0B1F930F9302
:1026500089EB98E00AC22D3091F4C72EDD24EE24D8
:10266000FF24B601112321F480E090E00E944E0B7C
:1026700080E591E09F938F937F936F93B8C0233051
:1026800009F570FF03C066EB78E004C071FF06C077
:1026900063EB78E0C5010E94CB1A17C272FF03C03A
:1026A0006AEA78E0F7CF73FF03C061EA78E0F2CF1F
:1026B00074FF03C068E978E0EDCFFF93EF9383E9FF
:1026C00098E0D3C1213191F0243081F0253471F0AC
:1026D0002E3261F02C3251F02F3241F0223531F0A0
:1026E000233441F0822F87548630C8F4C72EDD246E
:1026F000EE24FF24C701B60124E630E040E050E0BC
:102700000E942D1A2FEF30E040E050E00E94951A11
:10271000C901DA016C017D0185E290E0F1C025304C
:1027200041F02F3031F0263421F0822F8C53843049
:10273000C0F52C53243080F4C701B6012AE030E004
:1027400040E050E00E94951A285230406901EE2482
:10275000D7FCE094FE2C08C0872F90E088976C018E
:10276000EE24D7FCE094FE2CA601112381F49601FF
:1027700063E0220F331F6A95E1F72C0D3D1DC9015F
:1027800065E070E00E94601AAB01405E5F4F80918F
:10279000A00190E09F938F935F934F9388EE90E01A
:1027A00086C1223389F4CF0164E070E00E94601A90
:1027B0006B01EE24D7FCE094FE2C2CE231E03F9339
:1027C0002F937F936F9313C0822F8451883018F515
:1027D00085E0789F900111246901EE24FF249F3F3A
:1027E00049F48FE291E09F938F933F932F9386ED6F
:1027F00090E05DC184E6989FC0011124805092430F
:1028000060E870E00E94601A7F936F933F932F936C
:1028100089E898E04CC1822F8452883018F0223425
:10282000E9F402C0223421F4CF016AE070E003C071
:10283000CD0162E570E00E944C1A6B01EE24FF248A
:102840008E010F5E1F4F22E0A801C701B6010E9452
:102850005D0B1F930F938EEE90E007C1822F845380
:10286000883020F5BD0180E090E024E630E040E0D3
:1028700050E00E942D1A672F782F892F992787FD06
:102880009A95605870406B01EE24D7FCE094FE2CC2
:102890008E010F5E1F4F22E0A801C701B6010E9402
:1028A0005D0B1F930F9382E391E0DFC02434B1F4FA
:1028B000CF0168E471E00E944C1A6B01EE24FF2402
:1028C0008E010F5E1F4F22E0A801C701B6010E94D2
:1028D0005D0B1F930F9386E898E0C7C0213211F07B
:1028E0002133A9F4112349F4C701B6010E944E0B0C
:1028F000AC01CB01DA016C017D018091500190E0C7
:102900009F938F93DF92CF928CED90E0D0C02F31C8
:1029100031F5CF016CE370E00E944C1A9F938F93C6
:10292000CF016CE370E00E944C1ACB016CE370E0C5
:102930000E944C1A9F938F93CF0160E17EE00E942A
:102940004C1A7F936F9389E798E09F938F93BF9280
:10295000AF920E94E61A8DB79EB70A96B1C0822F39
:102960008D54823028F4FF93EF9382E798E07DC086
:10297000822F8650843010F02D32C9F48EE4789F77
:10298000C0011124805097426C01EE24D7FCE094E2
:10299000FE2C8E010F5E1F4F22E0A801C701B60179
:1029A0000E945D0B1F930F9382EE90E05EC0822F1A
:1029B0008A50823018F0233391F402C02A3019F083
:1029C000C72EDD2405C083E0789FC00111246C016F
:1029D000EE24FF24DF92CF9283EF90E046C02E30AA
:1029E00069F47695872F90E0805490406C01EE2436
:1029F000FF249F938F938EE698E037C02C31A1F48B
:102A0000C72EDD24EE24FF24723138F469E0769F6E
:102A1000B00111246857784F3DCE872F90E09F93E7
:102A20008F9385E698E021C0223249F5C701B601AF
:102A30002EE430E040E050E00E942D1A2AE030E021
:102A400040E050E00E94951AC901DA016C017D0155
:102A50008E010F5E1F4F22E0A801C701B6010E9440
:102A60005D0B1F930F938EE598E09F938F93BF921A
:102A7000AF920E94E61A8DB79EB7069621C04330EA
:102A8000510529F4C72EDD24EE24FF240AC0463068
:102A9000510539F49D01492F572FC901DA016C0105
:102AA0007D01FF92EF92DF92CF928AE598E09F93AB
:102AB0008F93BF92AF920E94E61A8DB79EB7089689
:102AC0000FB6F8949EBF0FBE8DBFB601C701A0968A
:102AD0000FB6F894DEBF0FBECDBFCF91DF911F912F
:102AE0000F91FF90EF90DF90CF90BF90AF9008953F
:102AF0000F931F93DF93CF93CDB7DEB7A8970FB691
:102B0000F894DEBF0FBECDBF8E010F5F1F4FB8011F
:102B100080E00E94BB126093A2017093A301809396
:102B2000A4019093A50160E080E20E943B118823FC
:102B300061F0B80180E20E94BB126093590170936A
:102B40005A0180935B0190935C0160E080E40E94F5
:102B50003B11882371F0BE016F5F7F4F80E40E94BC
:102B6000BB1260935D0170935E0180935F0190934F
:102B70006001A8960FB6F894DEBF0FBECDBFCF910F
:102B8000DF911F910F910895EF92FF920F931F9382
:102B9000DF93CF93CDB7DEB7A8970FB6F894DEBF1B
:102BA0000FBECDBF8C01F62EE42ECE0101962FED87
:102BB000261738F46EE0F69EB00111246755754073
:102BC00006C06EE0F69EB0011124615A7D4F0E944E
:102BD000CB1ACE0101966F2D70E0EE2039F07F9375
:102BE0006F939F938F9388ED98E006C09F938F9388
:102BF0007F936F9380ED98E09F938F931F930F9334
:102C00000E94E61A8DB79EB708960FB6F8949EBF3D
:102C10000FBE8DBFC801A8960FB6F894DEBF0FBED9
:102C2000CDBFCF91DF911F910F91FF90EF9008954D
:102C300080933E0160933F01409340012093410106
:102C400088E391E00E94E618089592E090933E0197
:102C500080933F01609340011092410188E391E02D
:102C60000E94E618089591E090933E0180933F0101
:102C7000109240011092410188E391E00E94E61811
:102C800008951F93CF93DF93EC0111E007C081E01B
:102C900090E00E941F0C1F5F1A3F59F00E947A18A3
:102CA0008823A9F31A3F29F0CE010E948B188111C5
:102CB00010E0812FDF91CF911F9108954F925F9285
:102CC0006F927F928F929F92AF92BF92CF92DF923C
:102CD000EF92FF920F931F93DF93CF93CDB7DEB7A1
:102CE0002E970FB6F894DEBF0FBECDBF8AE199E0F4
:102CF0000E944D0D0E94350DEE242E010894411CBA
:102D0000511C41EF642E43E3742E4BED842E48E1B9
:102D1000942E3FEDA32E37E0B32EC12CD12CEE2004
:102D200011F486E001C085E00E94F61780EE98E07D
:102D30000E94351900E0002361F4A0923801B0929E
:102D40003901C0923A01D0923B0180913C018D7FC4
:102D50000BC0609238017092390180923A019092D2
:102D60003B0180913C01826080933C0161E081E005
:102D70000E94251610E0FF24C2010E9441168823FC
:102D800009F040C088858134E9F589858130D1F525
:102D90008B858770843019F48C85882399F189811B
:102DA0009A81AB81BC81002321F40897A109B10964
:102DB0000AC0BA2FA92F982F8827A070B0708F5003
:102DC0009F4FA542B74E8093380190933901A0934D
:102DD0003A01B0933B01EE2019F484E199E002C07E
:102DE0008EE099E00E944D0D002319F487E099E0F0
:102DF00002C080E099E00E943F0D88EE93E00E94BF
:102E00001F0C11E0F39483E0F81609F0B5CF0F5FC3
:102E1000023019F4112329F008C0112309F48BCFD3
:102E200004C0E39481E0E8227ACF2E960FB6F8949E
:102E3000DEBF0FBECDBFCF91DF911F910F91FF90ED
:102E4000EF90DF90CF90BF90AF909F908F907F904A
:102E50006F905F904F9008954F925F926F927F9224
:102E60008F929F92AF92BF92CF92DF92EF92FF929A
:102E70000F931F93DF93CF93CDB7DEB72E970FB687
:102E8000F894DEBF0FBECDBF5C01EE24FF24CC243E
:102E9000DD243E010894611C711CE0E34E2E7AE0B3
:102EA000572E67E0862E912C8C0E9D1EC3010E942A
:102EB0004116882309F03FC00F81202F207F19F48D
:102EC000E02EFF2421C02031C1F4802F90E08F70CC
:102ED0009070F82EEE248885E80EF11C40923E0199
:102EE00010923F01509240011092410188E391E01D
:102EF0000E94E61806E082E008C02032E1F40E2DC0
:102F00000C19083008F007E081E010E095012C0D65
:102F10003D1DA401480F511DCA01402F50E0BC01C6
:102F2000C9010E94D21AC00ED11EEC14FD0409F092
:102F3000BDCF970102C02FEF3FEFC9012E960FB60C
:102F4000F894DEBF0FBECDBFCF91DF911F910F91DF
:102F5000FF90EF90DF90CF90BF90AF909F908F90B9
:102F60007F906F905F904F9008952A980E94271A43
:102F70008FEF0E94271A2A9A0895FF920F931F93AA
:102F8000182F062FF42E2A9885E00E94271A812FE9
:102F90000E94271A802F0E94271A8F2D0E94271A1D
:102FA0002A9A1F910F91FF9008951F93182F2A9826
:102FB00083E00E94271A812F0E94271A8FEF0E9418
:102FC000271A2A9A1F9108950F931F93182F062FDF
:102FD0002A9882E00E94271A812F0E94271A802FA8
:102FE0000E94271A2A9A1F910F9108950F931F93F9
:102FF000CF93DF93182F883008F055C02A9A229A71
:103000002D982B982C98259A239A24980E94221A5E
:103010002A9880EC0E94271A80EA9FE00197F1F736
:103020002A9A80E49CE90197F1F72A9882E00E94AD
:10303000271A88E20E94271AE3E01E9FE00111246C
:10304000FE01EA5DF64FE4918E2F0E94271AFE01E1
:10305000E95DF64F0491802F0E94271AC85DD64F74
:10306000FE0184910E94271A83E00E94271A2A9A5F
:1030700060E08DE00E94E41753985B9A68E08CE072
:103080000E94E41789E20E94D517182F60E08FE0B4
:103090000E94E417101739F48EE00E94D517807E45
:1030A000D9F781E001C080E0DF91CF911F910F91AE
:1030B000089540E060E48BE20E94BD1740E060E4C8
:1030C0008CE20E94BD1740E060E28CE00E94BD17D8
:1030D00082E00E94FE19089540E260E28CE00E94C6
:1030E000BD1740E460E48BE20E94BD1783E00E94BC
:1030F000FE19089589B1869586958695809581708B
:10310000089580EA0E94B51720E08475843509F09F
:1031100021E0822F0895CF92DF92FF920F931F93A9
:10312000CF93DF93EC0180EB0E94B517F82E082FA8
:1031300010E030E4C32ED12CC022D12286FF02C081
:1031400080E905C087FD02C080E038C084E92A9884
:103150000E94271ACE010E94AE198170880F2C811F
:103160002D7F282B2C838FEF0E94271A23E01695A2
:1031700007952A95E1F7302F31702C812E7F232B74
:103180002C83082F0F700D8310E008C08FEF0E9472
:10319000271AFE01E10FF11D86831F5F1017B0F3A0
:1031A0002A9ACD2819F040E061E002C040E062E0D8
:1031B0008CE20E94BD178F2D87708F5FDF91CF91BA
:1031C0001F910F91FF90DF90CF900895FF920F9382
:1031D0001F93CF93DF93EC0180EA0E94B51782FD25
:1031E00002C0FF240BC084FD03C032E0F32E06C0F2
:1031F00086FF02C0FF2433C024E0F22E2A988F2DD0
:1032000080640E94271A6C8166956170CE010E94CD
:1032100071190D810F702C8120FF05C0802F8064F3
:103220000E94271A0EC0802F0E94271A10E007C0A4
:10323000FE01E10FF11D86810E94271A1F5F101702
:10324000B8F32A9A25E02A95F1F72A98FF2011F47D
:10325000FF24F3948F2D80680E94271A2A9A8F2DBD
:10326000CDB7DEB7E5E00C94BD1A0F931F93CF9353
:10327000DF93EC0140E860EE8FE00E94BD178EE026
:103280000E94D517807E8038D1F764E080E60E94E6
:10329000E41760E080E70E94E41700E02A9882E0EB
:1032A0000E94271A802F0E94271A10E0003211F482
:1032B000183048F4FE012196E4918E2F0E94271ABF
:1032C0001F5F1C3099F72A9A005F003339F740E0FE
:1032D00060EE8FE00E94BD17DF91CF911F910F919B
:1032E0000895CF93DF93EC016623E1F02A813B81BF
:1032F00055E0369527955A95E1F72EBD2A810DB4F4
:1033000007FEFDCF3EB5822F880F880F880F807E85
:1033100088602370822B0E94271A89810E94271AB5
:10332000888117C02881398143E0369527954A95D1
:10333000E1F72EBD28810DB407FEFDCF3EB5822FEB
:103340008295880F807E0E94271A80E00E94271AAB
:1033500080E00E94271ADF91CF9108951F93CF93A9
:10336000DF93EC018FEF0E94271A182F8FEF0E9436
:10337000271A412F50E083FF21C02FEF2EBD35E0EB
:10338000440F551F3A95E1F75B834A830DB407FE5E
:10339000FDCF2EB529832FEF2EBD282F23703A8124
:1033A000232B8695869586958C71282B2A830DB4C0
:1033B00007FEFDCF2EB5288381E01CC02FEF2EBD68
:1033C0001B821A8223E0440F551F2A95E1F7598387
:1033D00048830DB407FEFDCF2EB52FEF2EBD82958D
:1033E000869587702881282B28830DB407FEFDCF92
:1033F0002EB580E0DF91CF911F9108951F93CF9359
:10340000DF93882311F410E609C0813011F410E431
:1034100005C0833011F410E201C010E0412F60EECE
:103420008FE00E94BD17C12FD0E08EE00E94D5171B
:1034300090E0807E90708C179D07B9F7DF91CF9157
:103440001F91089521E52CBD21E02DBD08958EBD6D
:103450000DB407FEFDCF8EB50895629FD001739F16
:10346000F001829FE00DF11D649FE00DF11D929F20
:10347000F00D839FF00D749FF00D659FF00D99275F
:10348000729FB00DE11DF91F639FB00DE11DF91F83
:10349000BD01CF0111240895AA1BBB1B51E107C038
:1034A000AA1FBB1FA617B70710F0A61BB70B881FD4
:1034B000991F5A95A9F780959095BC01CD01089563
:1034C00097FB092E07260AD077FD04D0E5DF06D04A
:1034D00000201AF4709561957F4F0895F6F7909546
:1034E00081959F4F0895A1E21A2EAA1BBB1BFD01D7
:1034F0000DC0AA1FBB1FEE1FFF1FA217B307E407D3
:10350000F50720F0A21BB30BE40BF50B661F771F2A
:10351000881F991F1A9469F760957095809590950A
:103520009B01AC01BD01CF01089597FB092E052633
:103530000ED057FD04D0D7DF0AD0001C38F45095C8
:103540004095309521953F4F4F4F5F4F0895F6F7C7
:1035500090958095709561957F4F8F4F9F4F0895FF
:103560002A88398848885F846E847D848C849B8413
:10357000AA84B984C884DF80EE80FD800C811B8121
:10358000AA81B981CE0FD11D0FB6F894DEBF0FBE50
:10359000CDBFED010895FB01DC0105900D920020E7
:1035A000E1F70895FB01DC0102C001900D9241504A
:1035B0005040D8F70895FC0161507040019001100F
:1035C000D8F7809590958E0F9F1F0895AEE0B0E0DC
:1035D000ECEEFAE10C94B81D0D891E892EE02C83C7
:1035E0001A8309832FEF3FE73E832D83AE01475EA9
:1035F0005F4F6F89788DCE0101960E94091B2F8144
:103600003885020F131FF80110822E96E4E00C9407
:10361000BE1AABE0B0E0EFE0FBE10C94AA1D3C0168
:103620002B015A01FC0117821682238121FD03C060
:103630008FEF9FEFC3C12AE0822E1E010894211C48
:10364000311CF3014381F20143FD859143FF8191D8
:103650002F01882309F4AFC1853241F443FD259140
:1036600043FF21912F01253231F485E2B30190E02F
:103670000E94201DE6CF322FDD249924CC24FFE1C7
:10368000FD15D0F03B3269F03C3228F4303259F06D
:10369000333291F40EC03D3249F0303369F421E009
:1036A00024C032E0D32A84E0D82A28C098E0D92A5E
:1036B00025C0E0E1DE2A22C0D7FC29C0232F2053F9
:1036C0002A3070F4D6FE05C0C89CC02C1124C20E4E
:1036D00015C0989C902C1124920EF0E2DF2A0EC0A7
:1036E0003E3229F4D6FC67C120E4D22A07C03C361A
:1036F00019F430E8D32A02C0383649F4F20143FD08
:10370000359143FF31912F01332309F0B8CF232F97
:103710002554233018F02052233038F424E030E0D0
:10372000A20EB31E3FE339830FC0333631F0333777
:1037300079F0333509F056C020C0F5012081298386
:1037400022E030E0A20EB31E710101E010E012C0D1
:10375000F501E080F180D6FC03C06FEF7FEF02C07F
:103760006C2D70E022E030E0A20EB31EC7010E9473
:10377000DB1A8C013FE7D32214C0F501E080F18011
:10378000D6FC03C06FEF7FEF02C06C2D70E022E02B
:1037900030E0A20EB31EC7010E94151D8C0130E857
:1037A000D32AD3FE07C01AC0B30180E290E00E9482
:1037B000201D9A94292D30E002171307A8F30EC09C
:1037C000F701D7FC8591D7FE81917F01B30190E08D
:1037D0000E94201D91109A9401501040011511056E
:1037E00079F7E6C0343611F0393651F5D7FE08C006
:1037F000F501608171818281938124E030E00AC00B
:10380000F50120813181B901882777FD8095982FB6
:1038100022E030E0A20EB31E0D2D0F7697FF08C0F8
:1038200090958095709561957F4F8F4F9F4F006861
:103830002AE030E0A1010E944C1DD82ED21840C0D1
:10384000353729F41D2D1F7E4AE050E01DC01D2D87
:10385000197F3F3661F0303720F4383509F0ABC0BE
:103860000FC0303739F0383709F0A5C004C048E040
:1038700050E00AC0106114FD146040E150E004C043
:1038800014FD166040E152E017FF08C0F5016081A9
:1038900071818281938124E030E008C0F5012081AC
:1038A0003181B90180E090E022E030E0A20EB31E49
:1038B0009A01A1010E944C1DD82ED218012F0F771A
:1038C00006FF09C00E7FDC1430F404FF06C002FDC1
:1038D00004C00F7E02C01D2D01C01C2D04FF0CC0B2
:1038E000FE01ED0DF11D2081203311F4097E08C089
:1038F0001F5F02FF05C003C0202F267809F01F5F5D
:10390000E02EFF2403FD14C000FF0FC0191510F0B6
:10391000CD2C0BC0CD2CC90CC11A192D06C0B3017A
:1039200080E290E00E94201D1F5F1915C0F304C0C3
:10393000191510F4911A01C09924E4FE10C0B301C6
:1039400080E390E00E94201DE2FE1EC0E1FC03C067
:1039500088E790E002C088E590E0B3010CC02E2D0E
:10396000267891F0E1FE02C08BE201C080E207FD03
:103970008DE2B30190E00E94201D06C0B30180E3F8
:1039800090E00E94201DCA94DC14C0F3DA94F10187
:10399000ED0DF11D8081B30190E00E94201DDD201E
:1039A000A9F706C0B30180E290E00E94201D9A941E
:1039B0009920C1F746CEF301868197812B96E2E1EB
:1039C0000C94B01ADC01CB01FC01F999FECF06C0C2
:1039D000F2BDE1BDF89A319600B40D9241505040CD
:1039E000B8F70895A8E1B0E042E050E00C94E41C80
:1039F000DC01CB0103C02D910E94031D41505040BA
:103A0000D0F70895262FF999FECF1FBA92BD81BD38
:103A100020BD0FB6F894FA9AF99A0FBE0196089550
:103A20000E94021D272F0C94031DFC01059061507C
:103A300070400110D8F7809590958E0F9F1F0895C4
:103A40000F931F93CF93DF938C01EB012B8121FF09
:103A50001BC022FF0DC04E815F812C813D8142172A
:103A600053075CF4E881F9818193F983E88305C009
:103A7000E885F9850995892B39F42E813F812F5FDF
:103A80003F4F3F832E8302C00FEF1FEFC801DF912E
:103A9000CF911F910F910895FA01AA27283051F173
:103AA000203181F1E8946F936E7F6E5F7F4F8F4F6F
:103AB0009F4FAF4FB1E03ED0B4E03CD0670F781FCE
:103AC000891F9A1FA11D680F791F8A1F911DA11DB3
:103AD0006A0F711D811D911DA11D20D009F46894EC
:103AE0003F912AE0269F11243019305D3193DEF694
:103AF000CF010895462F4770405D4193B3E00FD04A
:103B0000C9F7F6CF462F4F70405D4A3318F0495D34
:103B100031FD4052419302D0A9F7EACFB4E0A69517
:103B20009795879577956795BA95C9F70097610539
:103B3000710508959B01AC010A2E0694579547958F
:103B400037952795BA95C9F7620F731F841F951F84
:103B5000A01D08952F923F924F925F926F927F9295
:103B60008F929F92AF92BF92CF92DF92EF92FF928D
:103B70000F931F93CF93DF93CDB7DEB7CA1BDB0B39
:103B80000FB6F894DEBF0FBECDBF0994F894FFCFF7
:103B9000FF0232010A643464642100000000000066
:103BA0000000000000000000000000000000000015
:103BB00000000000E1E2E705E2E6E3E55061006DA8
:103BC00056002573206D4100000000000008555587
:063BD000555555555555F1
:00000001FF
